:020000040000FA
:100000008301262800000000F000030E8301F100A8
:100010000B1183120313A10F0E28A20AA30F11289C
:10002000A40AA90F1428AA0AAB0F1728AC0AAD0F0F
:100030001A28AE0A710E8300F00E700E09008B13A1
:100040008B1B1F2873088A007208820020308B00E7
:100050008312031300308500003086008F30831632
:1000600081003E3085009F308600831207309F005C
:100070008313203084008001840A841F3B28841667
:100080008001840AF0300402031D402883172030C9
:1000900084008001840A50300402031D4928831221
:1000A000031381010B118B17640083120313851D49
:1000B0005D28061C5D28201060288312031320147D
:1000C000201C6628A101A201A01473288312031327
:1000D000A01C73280F302202031C73284230210217
:1000E000031C7328A01083120313A01C7B28A01CE0
:1000F0007E2820157E2883120313201183120313F8
:10010000A01D8828201D8828201B882820168B28C1
:1001100083120313201207302402031D9128A130FB
:100120002302031C9E280730A402A130A302031C53
:10013000A403A0199D28A0159E28A01183120313C3
:10014000A018A428A501B22883120313201EB228E8
:100150002618B2282614A01AAF28A50AB22883129E
:100160000313A50383120313201AB7282610A01225
:100170002130F2000130F3002508F2070318F30ADA
:100180001F2083120313A7008B172718C9280510F7
:10019000CA280514A718CE288513CF288517271934
:1001A000D3280613D4280617A719D828A810D928A9
:1001B000A814271ADD282810DE282814A71AE228F8
:1001C000A013E328A017A01FE928A901AA0120175E
:1001D000F62883120313201FF6282D302A02031C51
:1001E000F628C7302902031CF628201383120313B4
:1001F000281CFE28AB01AC0105170B298312031341
:10020000051F0B293D302C02031C0B2909302B0242
:10021000031C0B29051383120313A81C1329AD011A
:10022000AE018616202983120313861E20292D3045
:100230002E02031C2029C7302D02031C2029861200
:1002400054280134043404341434183418341A345F
:020250003A343E
:084000000000010000000000B7
:02400E00543F1D
:00000001FF
